:0200000480007A
:1000000017180000130808001300100093001000D8
:10001000130110009301100013021000930210004E
:100020001303100093031000130410009304100036
:10003000130510009305100013061000930610001E
:1000400013071000930710009390F00163C40000A1
:10005000930000001311F10163440100130100003B
:100060009391F10163C40100930100001312F201A6
:1000700063440200130200009392F20163C4020081
:10008000930200001313F301634403001303000001
:100090009393F30163C40300930300001314F4016A
:1000A00063440400130400009394F40163C4040047
:1000B000930400001315F5016344050013050000C7
:1000C0009395F50163C40500930500001316F6012E
:1000D00063440600130600009396F60163C406000D
:1000E000930600001317F70163440700130700008D
:1000F0009397F70163C407009307000023200800CB
:10010000232218002324280023263800232848000F
:10011000232A5800232C6800232E780023208802ED
:10012000232298022324A8022326B8022328C802E7
:10013000232AD802232CE802232EF802971000006D
:10014000938040F01308100093081000130910006A
:1001500093091000130A1000930A1000130B1000EB
:10016000930B1000130C1000930C1000130D1000D3
:10017000930D1000130E1000930E1000130F1000BB
:10018000930F10001318F8016344080013080000CF
:100190009398F80163C40800930800001319F9014B
:1001A00063440900130900009399F90163C409002D
:1001B00093090000131AFA0163440A00130A0000AD
:1001C000939AFA0163C40A00930A0000131BFB010F
:1001D00063440B00130B0000939BFB0163C40B00F3
:1001E000930B0000131CFC0163440C00130C000073
:1001F000939CFC0163C40C00930C0000131DFD01D3
:1002000063440D00130D0000939DFD0163C40D00B8
:10021000930D0000131EFE0163440E00130E000038
:10022000939EFE0163C40E00930E0000131FFF0196
:1002300063440F00130F0000939FFF0163C40F007E
:10024000930F000023A0000123A2100123A420018A
:1002500023A6300123A8400123AA500123AC60014A
:1002600023AE700123A0800323A2900323A4A00344
:1002700023A6B00323A8C00323AAD00323ACE00322
:1002800023AEF003171500001305C5D7971500001E
:10029000938545DF370610F01306C6F26306B502F4
:1002A0008326C5002320D600832685002320D60080
:1002B000832645002320D600832605002320D60070
:1002C000130505016FF09FFD370510F0130505F2CA
:0402D00023200500E2
:10100000FFFFFFFFFFFFFFFFFFFFFFFFFFFFFFFFF0
:10101000FFFFFFFFFFFFFFFFFFFFFFFFFFFFFFFFE0
:10102000FFFFFFFFFFFFFFFFFFFFFFFFFFFFFFFFD0
:10103000FFFFFFFFFFFFFFFFFFFFFFFFFFFFFFFFC0
:10104000FFFFFFFFFFFFFFFFFFFFFFFFFFFFFFFFB0
:10105000FFFFFFFFFFFFFFFFFFFFFFFFFFFFFFFFA0
:10106000FFFFFFFFFFFFFFFFFFFFFFFFFFFFFFFF90
:10107000FFFFFFFFFFFFFFFFFFFFFFFFFFFFFFFF80
:040000058000000077
:00000001FF
